:020000020000FC
:100000000DC00AC0BBC308C095C306C094C304C0DA
:1000100003C002C001C0D8C3F894FECF32E04FE560
:100020003EBF4DBF002400270CBA00927F00009213
:1000300071000092720000927E003AEF3BBB32E406
:100040003ABB3CEF38BB37E037BB619A3BB7306116
:100050003BBF39E2A89531BD35E033BF31E039BF50
:1000600030E040ED3BBD4ABD3CE030936700479A2D
:10007000B1E0AEEF7AD64D3411F4393489F033E380
:1000800095D3F3E1E2E7B591BB2351F0A5913B2F66
:10009000B3703695369525917FD63A95E1F7F3CF33
:1000A00071D4789478E01CD233274427DE9A00007C
:1000B000CC9B0DC0DE980000CC9909C03A95B1F7F1
:1000C000A895442399F7439534E370D3EFCF4423A5
:1000D00011F0A9D49CC4D698DE9A44B743FD0FC052
:1000E0000092600000926600009261003DE2B0E084
:1000F000A7E84BE13D934A95E9F731E30AC0477F12
:1001000044BF30916100339509F43A953093610012
:1001100032E34CD311D130917F00353010F43030C0
:1001200009F47EC088D4323030917F0011F028F479
:1001300008C0323051F0A8F408C0323061F088F5C0
:100140000AC03230F1F0E8F46BC03091DC0036FFC9
:1001500067C05CE062C054E036D063E0B0E0ACE081
:1001600051C040918000439540938000B0E0A8E0EA
:1001700001D6431708F454C0B0E0A6E050E062E0B6
:1001800041C040918000439540938000B0E0ABE0D7
:10019000F1D5431708F444C0B0E0A9E050E061E0B5
:1001A00031C04091820043954093820000928000CC
:1001B00058E009D090F2B0E0AEE0DCD5409182008A
:1001C000431758F62DC0252FB0E0A3E0D3D5332335
:1001D000B1F044277AD36091D8005091D9003517F7
:1001E000460768F42FE0309185004091860035176E
:1001F000460728F4509385006093860001C08894D8
:10020000522F0895009280000092820060937F0038
:10021000ACD5409383003093840050936C0010D58C
:1002200031E1C4D20F70FEE0EAE2A6D004FD006224
:1002300016F433E1BBD230916600332319F03395C5
:100240003093660004FF13C030916000343018F41E
:10025000FEE0E2EB91D0FEE0EAEC8ED00F7E16F0ED
:10026000009260003091660033953093660006FD81
:1002700057D5F0917100E0917200FF2311F4EE2345
:1002800029F0009271000092720009953091660089
:10029000343610F053D0C4CF47E133273A95F1F705
:1002A0004A95D9F741D2A895532F30917E00432F1C
:1002B0004295341719F03517B1F7F7CF05FDB0CFD8
:1002C0005091830040918400A89531B5306431BDD0
:1002D00030E335BF889505FD2EC049505040A8F742
:1002E00030917F00353081F43AEF3BBB32E03ABBCE
:1002F00025D036E030937F00B0E0A1E136D54093C1
:100300008300309384008CCF30917F00363099F495
:10031000FFE0E6E131D008D202BA0ABA38EF0BBAF0
:1003200035E030937F00B0E0AFE01FD5409383000D
:1003300030938400C5CFEFCE33E008C033E03F9365
:1003400011C03F91332309F408953A953F93FEE09D
:10035000EEE000926C0010D040916C0040FF3F91A5
:1003600040FF0895FFE0ECE207D0319666D100929D
:10037000660074EBB5D0E5CF35E0932EF0936900BD
:10038000E0936A00F0916900E0916A00A8953491C9
:10039000303F29F43591359130936800F7CF313FE4
:1003A00019F43591EDD0F2CF332389F046D1FF9384
:1003B000EF93D1E0C32DE894B1D1C2D0E894FFE02F
:1003C000E2E4C4C0EF91FF919A94E1F66894089535
:1003D000EF91FF9134913323C9F60895006803C06B
:1003E0003FEF30936C00A8D0E9CFA6D08C2EAC2C78
:1003F00096D046F304FFE1CFAC1421F7C82D77D097
:100400001EF0FFE0E2EDA2D0E894D7CF04FF03C0D6
:1004100093D092D0D3CF23D0F0E1E0E897C0F0E0C2
:10042000E2EC02C0F0E0E2EA38E04081442321F04F
:1004300034963A9579F0F9CFB0E0ADE634E04D91DD
:1004400041933A95E1F706C0006130916000339521
:100450003093600071D063D0B1CF01D0AECF70D0F7
:10046000F0E0EDE634E00082D7D03EF0203328F013
:100470002A3318F421933A95B1F7089500625CD0BD
:100480009DCF5ED0F3E1E4E30B7F2CE2B22E7FD070
:1004900053D0B0E0A2EB38E0732EBB24FED14F93D3
:1004A0003F93B0E0AAEA38E0732EBB24F6D15F9107
:1004B0006F9124E0320F401D5317640708F4006465
:1004C0007DCFE2EC01C0E4ECF0E0BD2FAC2F34D0E6
:1004D00033E0732E3FEFB32EE0D1419331936ECFD3
:1004E000371711F0A895372F7723D1F70895E8949F
:1004F000B0E0A5E741E13ED44A958ED066F02032C7
:1005000029F02D3041F0231791F7F5CF332331F047
:10051000442321F0ECCF31E249D168940895332788
:10052000CC247AD096F02D3059F0303A28F4339517
:1005300030936500C226F5CF6FD03EF02D30E1F745
:100540006BD01EF02132E0F3CA9508958C2E759081
:100550007F9275907F927590772089F036F05CD00D
:10056000213618F02B3708F4205216F0271599F38E
:100570002F912F9175907720E9F7C82DE8CF089536
:10058000B0E0A2EA30E40D923A95E9F708953327F6
:100590007724AA24077F4591B591A5915B2FB3706D
:1005A0005695569539D0BEF12B1503FDD9F3077F2B
:1005B0002D3002FD2A32C9F0A226243211F402FDA8
:1005C000AA242B1559F402FF0860341729F4552387
:1005D00009F07C923395DFCF3395E4CF341721F4C3
:1005E000552311F02D935A95DDCF341719F4552367
:1005F00009F07C9202FF08950FD06EF020532A304C
:1006000008F027502295C22E07D02EF020532A3012
:1006100008F02750C20E089556F070916800C31577
:1006200041F4271711F0A895272F7723C1F7689475
:1006300008952991D1E0A895089532E0132E3591BF
:10064000373F28F43323B9F3232E4DD0F8CF3D3F65
:1006500058F53A3FA8F4383F58F43091630030938E
:10066000640000926300C090620000926200E7CFD5
:10067000B591A5914D91AC91B42F3170E7D0DFCFFA
:1006800055914591FF93EF93E0916B0030FDE09120
:100690006C0032FDEE27FF27EE0FFF1FE40FF51F62
:1006A000CEDFEF91FF91CBCF5527B591A5914B2F81
:1006B000B3704C7F632F3E3F38F42D90222089F099
:1006C00012D04450D1F7BBCF55D3232E222021F096
:1006D0000AD051604450C1F7560FA9F750E2252EB9
:1006E00002D0ADCF222E3F9330916300303A40F4D8
:1006F000339530936300309162003225309362006D
:100700001091670001600D7F02BA39E03EBD1123F0
:10071000F1F73F91089534E0132E02C031E0132E1B
:100720000E7F026012BA0895F89431E0132E0C7F08
:1007300012BA4EBC18955FB600FF0EC01A3011F009
:1007400030F427944BB2412808F041184BBA1A955F
:1007500009F40EBC5FBE189549B24120419427941C
:100760001A9551F40EBCFF93EF93F1E0E32D208234
:100770003394EF91FF9112BA5FBE18955FB649B2FC
:10078000412081F401FF10C02BB44AB42694479451
:1007900014E11419442442BA42084DBC1CBD19E0AE
:1007A0001EBD18E05FBE18950062FCCFA0917E00D0
:1007B000AF93A295A770AA58B0E03C93AF91A05F09
:1007C000A777A0937E00089578946FB6FF93EF9378
:1007D0003F93772309F07A953091750033953093E4
:1007E0007500E32F3F7039F430917300339509F4AD
:1007F0003A9530937300E0FD24C0E1FBE0917E0068
:10080000FE2FE295F770E770FE17D9F0E6E7EF0FDD
:10081000F0E0308166F4303120F0C19A30513083FD
:1008200010C0332371F0C09A315030830AC0C19890
:10083000C098332331F430917E003395377730936D
:100840007E003F91EF91FF916FBE1895FF93EF935C
:10085000F8E0EEE820E345914E3FB1F060F45591A9
:10086000A41BB50B18F023953260FACFA40FB51F67
:1008700031FD38DFEFCF313011F420E333DF326068
:100880002EE230FD2FDFE6CFEF91FF910895102784
:10089000E80364000A00FF0100FEE89433274427C0
:1008A0002D91BB2011F42E3269F02B1511F46894B0
:1008B00009C0205348F02A3038F407D05527320FAA
:1008C000451F16F07A9461F70895330F441F632F84
:1008D000542F660F551F660F551F360F451F08957D
:1008E0004FDEF0E1EAEA0B7F20E2B22E50DEF0E0CC
:1008F000E2EAB0E0A5E830E121914ED23A95E1F785
:100900007AC015D001C077D01BDEB0E0A5E130E29F
:1009100037D2B0E0A5E380DE4EF0203228F009F0B7
:10092000FACF30E42DD202C0222736D2089546E015
:1009300035E163C025DEF0E1EEEA0B7F20E2B22E66
:1009400026DEB0E0A2EAF0E0E2EB30E14D91519119
:10095000451791F4442311F03A95C1F73E3060F405
:10096000F0E0E2EAB0E0A5E730E1219115D23A9556
:10097000E1F746E03CE241C046E03EE23EC046E0F0
:100980003AE23BD033E03093830034E83093840084
:1009900030E030937F00089500928300009284003D
:1009A000009285000092860034E030937F0030EFA3
:1009B000309380003093820008950092830000926B
:1009C000840036E030937F0016C0F3E1EEE405C00A
:1009D000F3E1E6E502C0F3E1E6E6EAD146E032E320
:1009E0000CC0AADD46E030E308C045E032E005C0B7
:1009F00045E033E002C046E03AE2409371003093B4
:100A00007200089510D026D174EB6ADD97DCF8945B
:100A1000A89542E030E0F0E0E0E601923A95E9F78F
:100A20004A95D9F7FBCAB1E0AEEF2227B5D1B4D1D0
:100A30000895F894FECF0092DC0000927300C298F3
:100A4000D1E0C32D3CE3309368009ADD64DEA895C5
:100A5000F2E1E8EFE8947ACD16F06EDD18C030E0F0
:100A600099C0F3E1EEE002C0F3E1EAE2C82D0460D0
:100A70002CE2B22E8CDD64DD96F3AC1441F430919F
:100A8000A200313421F43091D000313370F4B0E061
:100A9000A1E040917F00413009F4A2E06BD1409188
:100AA00073004317A0F231E075C03091DC0033953C
:100AB0003093DC003F733A3050F3B0E0A1ED32E008
:100AC000732E3FEFB32EE9DE343060F440917F00A7
:100AD000413041F0B0E0A0E04DD1409173004317A8
:100AE00008F4D5CF3091C400332329F430E3309398
:100AF000C4000092C50030917F003330E8F4B0E0CC
:100B0000ABEAF0E0EFE855D060F4B0E0A6EBF0E03F
:100B1000EAE94FD030F43091DC003F7B3093DC00C9
:100B20000BC03091DC0036FD07C03064307C309360
:100B3000DC00009273008BCFB0E0A3ED35E0732EA4
:100B40003FEFB32EAADEB1EDA9EF5ED0F093DA004D
:100B5000E093DB00B0E0AEEB36E0732E3EE2B32E66
:100B60009CDEB3E9ADE452D0F093D800E093D90015
:100B7000B0E0A4E0FAD0FF2351F4E31740F4E41707
:100B800040F03091DC0037FD02C03068CFCF33E059
:100B900001C032E030937400C29A323048F0B0E0C5
:100BA000A3EAF0E0E7E84BE15D9151934A95E1F764
:100BB0000895FF93EF9356E0752EBB246EDEAF9140
:100BC000BF914F933F9356E0752EBB2466DE5F9135
:100BD0006F913517460728F0351B460B532F642FAE
:100BE00002C0531B640B45E730E35317640730F032
:100BF000352F462F6AEE50E6531B640BB0E0A3E19D
:100C0000B4D0531764070895330F441F330F441FA4
:100C100050E1FF27EE27B695A79510F4E30FF41FD8
:100C2000F795E7955A95B9F7089530917F003530DB
:100C300018F4303009F001C0FEDE34E130936C006E
:100C40004091740036E24030D9F137E34130C1F1D0
:100C500038E436C030E034C039E032C032E130C070
:100C60003EE12EC08DDCD0E0C2EAF3E1EEE42227C3
:100C70005591552399F0B52FBF70A5917BD044278E
:100C800055FF04C0330F441F330F441F57FF4993D0
:100C9000399357FFEDCF6ED03993EACF23952230A9
:100CA00021F030F4F3E1E6E5E3CFF3E1E6E6E0CF6F
:100CB0000992309161003993FEE0E6E95DDB3EE7A1
:100CC00030936B00B0E0A5E155D0332319F434E143
:100CD0006DDD25C033E030938100F0E1E6EB4CDBC5
:100CE000E6F0FEE0E2EB48DBC6F0AC1431F4309104
:100CF000640040916500341741F0FEE0EAEC3CDB13
:100D0000309181003A9549F0E6CF0F77F0E1EEEDB2
:100D100033DB1EF007FD04D0089532E147DD08956E
:100D2000FEE0E2EE29DBF0E0E2EA0068B0E0ADE6EA
:100D300034E041914D933A95E1F730916D003323C2
:100D400089F0FF93EF93E23C06FF20F0FEE0EAEC2F
:100D50000F7B05C007FF04C00F77F0E1EEED0CDB61
:100D6000EF91FF91EA3D10F30895BFBBAEBBE09A4F
:100D70004DB31196BFBBAEBBE09A3DB3119608953B
:100D80004BDC2EF0213218F007D03A95C9F7CA95FE
:100D90002227332309F40895BFBBAEBB2DBB2FB769
:100DA000F894E29AE19A2FBFE199FECF1196089547
:100DB000FF93EF93E5DBF3E1E4E30B7F20E2B22E58
:100DC000E6DBEF91FF91B0E0A2EABF93AF933C91D5
:100DD0003323D1F038E0732E3FEFB32E5EDD559113
:100DE000552391F0B52FBF70A59155FF04C04695CE
:100DF000379546953795242F57FDCEDF232FCCDF2F
:100E0000AF91BF911896E1CFAF91BF910895F008CF
:100E10001A415445300D00415445300D00F0144145
:100E2000542B4346554E3F0D0000F00841544530C9
:100E30000D00F01441542B434D47463D310D004108
:100E4000542B434E4D493D322C312C302C302C301C
:100E50000D00F141542B43504D533D224D45222C62
:100E6000224D45222C224D45220D0041542B434D4D
:100E7000474C3D225245432052454144220D0041FA
:100E8000542B434D474C3D2252454320554E52452D
:100E90004144220D0000F008415445300D00F0148B
:100EA00041542B4342430D0041542B4353510D00F9
:100EB0000000F008415445300D00F01441542B431C
:100EC0004D47523DFD106D0D0000F0084154453076
:100ED0000D00F01441542B434D47443DFD106D0D62
:100EE0000000F008415445300D00F141542B434DB2
:100EF000474C3D2253544F20554E53454E54220DDE
:100F00000041542B434D474C3D2253544F205345F1
:100F10004E54220D0000F008415445300D00F07889
:100F200041542B4346554E3D300D0000F0084154CE
:100F300045300D000041542A535752455345540D36
:100F40000000E2014552524F520D00E8014F4B0D97
:100F500000F0012B4346554E3A203000F3012B435D
:100F600046554E3A203100EE012B434D53533A0083
:100F7000F3012B434D53204552524F520041022B57
:100F800043504D533A002D022B434D47573A00062C
:100F9000022B434D474C3A00F5012B434D47523A43
:100FA000003E022B434D54493A00E8013E200061C7
:100FB000022B4342433A20302C0061022B43424330
:100FC0003A20312C0063022B4353513A2000E201B6
:100FD0000000830453455441444452455353007028
:100FE000045345544E414D45009A045345545041D5
:100FF0005353574F524400E804534554545241430D
:101000004B00EB04534554504F57455200E50453F1
:101010004554535045454400EE04535441545553F0
:101020000097044C4F4341544500810453414C4FB9
:101030004341544500BF04545241434B4F46460080
:10104000CC04545241434B4F4E00DD04504F5745A2
:10105000525341564500BF04504F5745524F4E0022
:10106000F8045245424F4F5400F5045245494E4949
:1010700054001905434155534557445200F10400AB
:101080000C022C000C0222000F0253544F20534537
:101090004E5400120253544F20554E53454E5400A7
:1010A000240252454320002A02000140A2FF0140D1
:1010B000A20240B2FF00F008415445300D00F01488
:1010C00041542B434D47573D22FE8015220D00F71A
:1010D000FF0035FF4085FA10F6F71A0D0000F00802
:1010E000415445300D00F07841542B434D53533D4E
:1010F000FD106D0D0000434F4D4D414E44204558AD
:10110000454355544544000050415353574F5244B2
:10111000204348414E474544000050415353574FE8
:101120005244204348414E4745204641494C45449E
:101130000000554E4B4E4F574E20434F4D4D414EA4
:1011400044004E4F204441544153545245414D2098
:1011500046524F4D2047505320444556494345FC85
:1011600012BC00004750532054494D4544204F5570
:10117000542057414954494E4720464F5220464932
:1011800058FC12BC0000FB128C20504F5320FD086D
:10119000A920FD1CAB20FD04B220FD0CB320FD1CDA
:1011A000B620FD04BD20414C5420F800DA204654FE
:1011B00020535045454420F900D8204D5048204345
:1011C0004F5552534520FD18C420415420FD08CEF0
:1011D0002FFD08CC2FFD08CA20FD08A33AFD08A565
:1011E0003AFD08A720555443205341545320FD088D
:1011F000D1005350444C4D543DF800A22053544F5D
:1012000050443DF800A82FF800AA20424C4B443D22
:10121000F800AC2FF800AE204D4F564E473DF80079
:10122000B02FF800B2205053563DF800B62FF8000A
:10123000B82033442F4649582F424C4B443DF800C8
:10124000BA2FF800BC2FF800BE204D442F4D533D5F
:10125000F800B42FF800A42FF800A6204241543D16
:10126000F800C2205349473DF800C4205744523D7E
:10127000F800C020563D302E3137204F70656E206B
:1012800047505320547261636B65720053544F5042
:101290005045440053544152544544004D4F564923
:1012A0004E4700004D4F5645440053504545444974
:1012B0004E4700004C4F4341544500002C204C4108
:1012C000535420474F4F442046495820FD088D2055
:1012D000FD1C8F20FD049620FD0C9720FD1C9A20FC
:1012E000FD04A120415420FD08873AFD08893AFDFC
:1012F000088B2055544300003105244750524D437C
:10130000003405244750474741002C0500000118D0
:10131000A30204A20324A90404B20528B30604BD51
:101320000718BE0818C40918CAFF0604D00708D158
:101330000914D3FF0120A20220AA0320B20420BA7C
:101340000520C20620CA0720D20820DAFF00400389
:10135000400440050000800640088009400B800CD6
:10136000400E80130000800F801120002001200219
:1013700000001075475053000485000435005400E8
:101380001222180014640078020258020078050E38
:1013900010025800C804150004350009FE4D49002C
:00000001FF
